:10000000E220A001AE017820AD00FF30850086001F
:10001000831606309F007F308100FF3085004F300F
:10002000860083120B30A9001830FA005830F9000E
:100030009E27BC20A90B18280530F70070308400DB
:100040007E20E2208A15CC24031D31287008CA3A8C
:10005000031D31287108213A03195629013A031961
:1000600056296A3A031D94287108A43A0319A22A52
:10007000843A0319A32F903A0319C42B703A031939
:100080002D2B163A0319C42B243A0319272B403A77
:100090000319D72B6E3A0319D72B543A0319F62EAE
:1000A000723A03199828D63A0319A52F083A03196A
:1000B000A72F863A0319622AB23A03196A29023A2B
:1000C00003197429063A0319AD29D63A03192B2AC4
:1000D000F03A0319382A363A0319A92F403A03197E
:1000E000A92F623A0319AB2F0E3A0319AB2F9628AA
:1000F000FF34E2207108BC2830308400AA20800040
:10010000840AF70B7E2808006B30A2286730A228EB
:10011000F001F22A0230F000F22A0830F000F22A50
:100120005030F0009830A3286E30A2286D30A228FD
:100130002E1DA1288A15BE2177086507F000913091
:10014000A3289030F001A300E2202308BC2070080F
:10015000BC201C28861BAA282830E5200930A100D5
:100160000310861F0314A20DE420A10BB028A20CDB
:100170002530E52022080800A300A200A209A00162
:100180003230E5208316861383128613A0170830B9
:10019000A100E42022088039A00606068606A20DEA
:1001A000A10BC928E420200806068606E420831651
:1001B00086178312E420861FE0282E30E5200800F1
:1001C0002308BC283B30E5281A30A400A40BE628FD
:1001D000003486160616000006120000861208007B
:1001E000031C061203180616861600008612080065
:1001F00083160616831286160310061A0314861237
:1002000008000830FD00FE0DF020FD0B0329F8204A
:1002100083160612831208000830FD00F820FE0D38
:10022000FD0B0E290829E920A030FE0001217A08E3
:10023000FE0001217908FE00012106122F21E9208C
:10024000A130FE00012108000C210310F0207E08DF
:1002500008000C210314F0202F217E08080006124C
:1002600000008616000006160800A100E920A03054
:10027000FE0001217A08FE0001217908FE0001211B
:100280002108FE00012106122F21E920A030FE00E6
:1002900001212F210318452908003521F90A0319E6
:1002A000FA0A0800F9070318FA0A08007208FA00A7
:1002B0007308F900213071020319512C7920740858
:1002C000F7007C203030840000084D21840AF40BB4
:1002D000642998287920AA20F40B6B29FE30E300CA
:1002E000E5018A15D424982879208A15BE218A151B
:1002F0009D23031999291F3A031D81298A15C925B0
:100300008A29C83A031D8D29AE126408AD008A15EA
:10031000DA21A5268A15BE2197298A1549230319B2
:100320009929013A0319AE15033A0319AE15B12301
:10033000AE112E119828A6219E27BE00E50783172F
:100340009E278000840ABE0BA02908001730FA00FF
:10035000AE30F9001130BA23080079208A154B25F8
:100360000318282A8A1556253B08FC39031D9828AE
:100370003308213A031DC229C9303202031D9828CF
:100380001630CC29053A031DFD292030E1003E0836
:10039000E3000319282AE4008A1524230319262AD6
:1003A0000A306302093C031CDA29CC30E3000A302E
:1003B000E402262A6308153A031DE129CB30E30045
:1003C000262A8A15AB240319262A043A031DF72985
:1003D0002D08303E0317A0002930A1002030A200D4
:1003E00003130330E500233084009B21262A3F3A83
:1003F000031D262A8A152224262A073A031D982837
:100400003208E300CB3A031D082A8A159122262AD6
:10041000DE3A031D0E2A8A15C122282ADD3A031D61
:10042000142A8A15E522262A8A15AF230319262ABB
:10043000C83A031D1E2A8A15F223262A0F3A031DE5
:10044000242A8A150224262A8A150C242E1E2E15EB
:100450002E12831398287920AA20F40B2C2A2E1907
:10046000282AE300013A031D272A8A15E424272AB3
:1004700079207408F700333084007E20AD270230E5
:10048000522113212421B0002421B1002921350754
:10049000B200031C512AB10A031D512AB00A0319E4
:1004A00090283408B107031C582AB00A0319902871
:1004B0003308B007031890288A15FD212E14063042
:1004C000F000CA2A79207408F7007C202608F4225C
:1004D00003198828013070079A27A400023070079A
:1004E0009A27A1000B3070079A27A30073080F39D1
:1004F0000319AC01AC0A2C08F6002308832A522108
:10050000A102031CA403F60B7F2AA408031D8B2A57
:10051000A1080319F02A1321292130060319972A6B
:1005200023085221AC0AA102031CA403852A7308E4
:10053000103903199828AE140130F000CA2A2C088B
:10054000BC20982872087304031D842802307402AA
:10055000031D862879200230F7007C203F303002CE
:10056000031DCC2AB108031DCC2A1630F000300838
:10057000A9003108AB003008A5003108A600AC0185
:10058000AC0A13212421D9002921D8008A1505227B
:100590002E10AE109F30A3287F303002031DDC2ABE
:1005A000103031020319B52A203031020319B52A5F
:1005B000213031020319B52A6F3030020319E82ABD
:1005C0002F303002031DF02AE2303102031DF02AE1
:1005D0003108A600AD270319F02A0F30F000BB2A1E
:1005E0000430F0009430A328F0001830FA00633093
:1005F000F9000430DC006A30DB009E27FF39031964
:10060000262B700603191D2B9E27F500F6019A274D
:100610002039031D0230F6007508013EF5009A27C7
:10062000013E0319FD2A750A9A277607DB0703188E
:10063000DC0A75089A27DC07FD2A9E27F0005C0873
:10064000FA005B08F90070089A27031108002908CE
:10065000A8002B08AA007920362B2508A800260818
:10066000AA0079202E18512BAE189F2A3F3028025D
:10067000031D3D2B0130F0005B2B7F302802031D52
:10068000442B1130F0005B2B6F3025020319712BC6
:100690002F3025020319712B0301BC20F40B4C2BC6
:1006A00098288A15A225303084000008BC20840ACE
:1006B000F40B552B9828F500F70105307702031D40
:1006C000632B2A086B2B10307702031D692B213016
:1006D000F50075089A27BC20F70AF50AF40B5D2B84
:1006E00098282608F422F600F00A8530BC200D3048
:1006F000BC2070089A27013E0230031D832B0301A2
:10070000BC20F00A0130F700AA2304307402031958
:1007100098282508BC202608BC200430760203193E
:10072000952B06307402F700A82B0430BC20003053
:10073000BC200130F700AA2309307402F700260814
:10074000073A0319A82B793A0319A82B2730F00090
:10075000AA23982870089A27BC20F00AF70BAA2B26
:1007600008009E27AE1DB62BA53A7906BC20F70BD4
:10077000B12B0800F6002D08F7000319C32B7608EB
:100780005221F70BC02B08002608F42203198D28EC
:10079000043A031D8D288A154E220319A328AD277C
:1007A00073085221D630710203195D2C512C260892
:1007B000F42203198D28043A03198D2820390319CE
:1007C000132CAD27F303F3030319F02BF3030319E1
:1007D000F62BF30B8D28720803190130AC00FF2BA8
:1007E00058082C020319AC01AC0AFF2BAC03DC3017
:1007F00071020319AC015808AC080319AC002C08AD
:10080000FF3E5907F600580876020319092C031811
:10081000F600DC307102031D102C7608D90035215A
:10082000023052212A2C8A1550220319A328AD2701
:10083000F303F3030319272CF3030319252CF30BFC
:100840008D287208031DAC00282CAC03282CAC0AA0
:100850002C08F600013070079A27A400A41BA40AF4
:10086000023070079A27A1000B3070079A27422C9C
:100870005221A102031CA403A408031D422CA108B9
:1008800003198A28F60B382C3A302602031D4C2C0B
:10089000FA1F4C2C8A15F52EDA01DC30710203198F
:1008A0005D2C79201321740303195A2CF40324219D
:1008B000BC20532C2921BC209828DC307102031D58
:1008C0006F2C3C302602031D6F2C7109BC20AA201E
:1008D0004D215A1C7924F40B652C2E1298288A1568
:1008E0001927A030840000084D21840AF40B732CD2
:1008F00098288A153D2103182B2E0319802C0800F7
:100900007C08F500A03084000830FB003030000285
:10091000031C2B2E3A30000203182B2E0F308005BB
:10092000AF263D26031C972CFB0B862C2B2E0F305D
:100930000005E200AF263D26031CF42C8403F50AD3
:100940000230FB002D2603182B2E8A159E21840AC7
:10095000840A3D260318C62CE20803192B2E6430A6
:10096000620203182B2E0008533A031D2B2EAF26CC
:1009700000084D3A031D2B2EF503031D2B2E0430CA
:100980008402620880005330E2005B2D0130FB00DE
:100990002D2603182B2E3D260318EF2C1A30620249
:1009A00003182B2E84038A159E21840380000430B3
:1009B0008407E20803192B2EFF30620203182B2E46
:1009C0000008413A031D2B2EAF260008443A031DB0
:1009D0002B2EF503031D2B2E4130E2005B2D05303D
:1009E000FB003230E200382D8403840330300002F3
:1009F000031C2B2E3A30000203182B2E62088000B5
:100A0000840A840A0008453A031D252D840A00083B
:100A10004E3A031D2B2EF503F503031D2B2E620802
:100A20002D0603192B2E7820620603192B2E840322
:100A30004530FB000F308000840AFB0B1B2DA030DB
:100A40000402FC005030E2005B2D5030E2006326CF
:100A500003182B2E3D2603182B2E712603182B2E40
:100A6000F50803195B2D3D2603182B2E0830FB00DB
:100A70002D2603182B2E3D2603182B2E0430FB00A9
:100A80002D2603182B2E0430FB00F5080319592DD1
:100A900030300002031C2B2E3A30000203182B2E9C
:100AA0000F308005AF26FB0B452DF50803195B2D94
:100AB0002B2E203080007A08DC007908DB002D081E
:100AC000DD007C08F500A030840045260318252EA3
:100AD000AF2653306202031DAD2D0008E200F50081
:100AE000DF01DE014430E1002F30E000B030DE07EE
:100AF0000318DF0AE002031CE103E20B762DA630A7
:100B0000F9000830FA00D0265F0603198B2D621415
:100B10005F08FB00DF264E21D0265E060319A22DBA
:100B200062145E08FB00DF26621CA22D8A30F900E9
:100B30000830FA006108FB00DF264E216008FB0048
:100B4000DF26202E7130F9002230FA000301352112
:100B5000B0305221F50BA62D202E41306202031D2C
:100B6000D42D0008E000E1010530E2000310E00DA3
:100B7000E10DE20BB72D8E30F9000830FA00D026D7
:100B800061060319C72D62146108FB00DF264E21A0
:100B9000D02660060319D02D6008FB00DF26202E2A
:100BA0006218202E2E16252E32306202031DDB2DF8
:100BB000F430F800FD2D0008AD00840A840A0730E7
:100BC0008A15AC210930FB00000E840A0007840A54
:100BD0004D21FB0BE42D840A2D0E003EF800103051
:100BE000FB009C263530F50203191A2E840AC83002
:100BF000F9000430BA237908F8000430FB009C2681
:100C0000840A32306202031D082EF030F8000E2EE6
:100C1000A030F9000430BA237908F8000430FB0052
:100C20008B267F08BD26F80AFB0B102E323062029D
:100C30000319D22DA5262E165D082D02031D252E83
:100C4000CC30E3005D08E4002E155C08FA005B0878
:100C5000F9005D08AD005A14080030300002031C92
:100C60003B2E3A30000203183B2E0F308005AF2692
:100C7000FB0B2D2E08000314080003140008203A73
:100C8000031D442EAF26031008000230F3008A151E
:100C9000A6268A11803A03193B2EF030F800043062
:100CA000F7008B26B226F80AFF06031D602EF70B0D
:100CB000512E8330FB060319432EFB00DF26432E03
:100CC000FB03DF263B2E0008303A031D3B2E840A2F
:100CD0000008383A031D3B2E84031230FB002D26FA
:100CE00008002030FB0030300002031C3B2E3A305D
:100CF0000002031C852E41300002031C3B2E4730AE
:100D0000000203183B2E373080020F308005AF26DB
:100D1000FB0B732E432E0008203AF0300319922E5D
:100D2000000EAF26FF000008203A0F3003199A2E5C
:100D30000008AF26FF070800000E840A0007840A97
:100D4000BD26F80AFB0B9C2E08007E308A15AC21CC
:100D50000B30FB00FF304D21FB0BAA2E0800840A4C
:100D6000F50308000317831278088D0083168C138F
:100D70000C1483120C0803130800031783128C0051
:100D800078088D0083168C130C1555308D00AA3011
:100D90008D008C140C118C18CB2E031383120800B9
:100DA0000317831279088D007A088F0083168C1739
:100DB0000C140000000083120C08FB00CD2E03175A
:100DC000831279088D007A088F007B088C003430FC
:100DD0008E0083168C170C158B1355308D00AA309E
:100DE0008D008C14000000000C11CD2E1030740208
:100DF000031D86282E1479207408F70040308400E3
:100E00007E200730D000303084001030F7002D0EE7
:100E1000003EF800B2268000F80A840AF70B0A2F79
:100E20000430F7000130D5001030D400D60155034E
:100E3000F6005403F50075085607D100303E8400D3
:100E40000008D200540884070008D3005208C727BE
:100E50008A018000540884025308C7278A01800051
:100E6000F503F51F1B2F0310540DD607F603F61FCD
:100E7000192F0310D50DD40CF703F71F162F3030A0
:100E800084000230F5001030F700000E840A0004E0
:100E9000F600840A750884027608800075088407C5
:100EA000F50AF70B452FD00803197A2F1030F700F9
:100EB0004030D200F5018030D5000830F600D10175
:100EC000750DD400D40E0F30D40530305407840093
:100ED00000085505D1040310D50C1130F507F60BA9
:100EE000602F5208840051088000D20AF70B5B2F54
:100EF000D003032F0230F6003F3084000730F700A4
:100F00000310800D8403F70B812FF60B7C2F073025
:100F1000F700393084000008F600053084027608B6
:100F2000800006308407F70B8B2FBB018A010C3041
:100F3000F000CA2A8A018A150020842D8A150D2105
:100F40008A014E2108008A15862D8A15042E8A15DD
:100F5000362E8A15D92E8A15BA2D8A15AB2900008E
:100F60000000000000000000000000000000000081
:100F70000000000000000000000000000000000071
:100F80000000000000005708530752070800D70070
:100F900007308A007708CD2782008207EF34E934D2
:100FA000E434E034D3345708D70153070318D70A81
:100FB00052070318D70AD7105706A1001030FD2F8B
:100FC000C327A1001130FD2FC3277F39A1001230A4
:100FD000FD2FC3273F39803EA1001230FD2FC327CC
:100FE000F900790C0F39C03EA1001230FD27FA003C
:100FF0007918FA0E7A0E0F3908008A00210882004B
:10100000820085341434003400343F340034013419
:10101000003404340034003400340934113404340E
:10102000033485341434003400347F3410340234F3
:1010300000340434003400340034093411340034F2
:1010400011340834003483348A3483348A34F034DD
:10105000443403340234003400340434003404349F
:1010600001340434FF3409341B34FF341B3401349D
:101070000234003400340434FF340B341134FF34B0
:101080001B3401340234003400340434FF34093496
:1010900011340434FF34103411340434003418345F
:1010A000113404340034013414340434FF34033470
:1010B0001234043400340A3414340434FF34053454
:1010C00012340434003402341134043400340A3449
:1010D000113404340034113404340434FF3409343A
:1010E00011340434FF340E34113404340034023427
:1010F0001434043400340C34113404340034033414
:1011000004340434003401340434043400340A3424
:101110000F34043400341F340F3414341F34C034FB
:10112000043400341134F0342234013402340134F4
:10113000203414341B34C034043400341234F034FA
:10114000443401340234013420341434443410342F
:10115000043400341134F0344434013402340134A2
:10116000B034143400341C34043400341134F034FA
:1011700044340134023401340E34143400347034F5
:10118000043400341134F034443401340234013472
:101190001C341434FF342034043400341134F0345B
:1011A00044340134023401342034143400344134E2
:1011B000043400341134F034443401340234013442
:1011C0000D34343401341834043400341134F03420
:1011D00044340134023403341C343434FF340334D3
:1011E00004344034123410344434013402340334AF
:1011F0000334303084002F08F9002708FA000F303C
:10120000F4000008840A8A114D218A15F40B012983
:101210007908AF007A08A700842D7A088A00790837
:1012200082008A1152218A1508008A11DF2E8A1144
:10123000AA208A1508000D218A014E218A1508006E
:101240008A112D268A1508008A11BA238A150800EA
:101250002030E000A030E2005030F6008317600834
:1012600084000008DD008313620884005D088000AC
:10127000E00AE20AF60B2E2908002208DA184629AD
:10128000F501073A031D9C29DA1499295A195329A3
:10129000F508031D4F29F504031951299929F50B68
:1012A00099295A159929DA195A29183903195A17F7
:1012B000DA1599295A1A5E295A169929DA1A6E29C5
:1012C000F508031D6A29F500F50A0310F50C033033
:1012D000F5079929F50B9929DA1699295A1B7229CC
:1012E0005A179929DA1B8629F500FC0009302202D9
:1012F000031C9C295130220203189C29A030FB00BA
:101300000830DB000730DC00DA179929DD00DD0C3E
:101310007B088400800CDC0B95290310800C0730BF
:10132000DC00FB0AF50303199A29DB0B8729083037
:10133000DB0003110310842D0314842D62080310B5
:10134000E20DE20DE20DE207E20784030008620706
:10135000E2008403842D2608E0001730FA0085306F
:10136000F900C4218A150319BA2977088A11BA230A
:101370000311080026088A11F42208006308E0001F
:101380001730FA001930F9001B2100380319842D99
:1013900060060319CE2903301121C4291B21A400A2
:1013A0001B21A1001B21F7002408FA002108F900E5
:1013B0000311842D0430FA00A930F9000C30FB0031
:1013C000FF308A114D218A15FB0BE0299925E50193
:1013D000203084009B210630FA006030F900203074
:1013E000840000088A114D218A15840AE50BF12931
:1013F000FF308A113521831308008A1130084D21EE
:1014000031084D2132084D210800AE1A832DAE1649
:101410008A110530FA004630F900132129218A1576
:101420000A3A031D122A8A114030FA00F9011321E9
:101430002421E5002921A30025084D212608352176
:10144000FA01F90113212421FB002921FC008A154E
:101450004030FA0065088A114D21230835218A158C
:101460007B082506031D382A7C0826060319372A1F
:10147000AD1FDA210830FA009530F9008A11D02624
:10148000A3003730F900D0262306031908002308EB
:10149000FB00DF264130F900DF2608000330512A27
:1014A000053070078A119A278A15F039031D5D2AC5
:1014B0007108F039D03A031D642A2D08FF3A031D44
:1014C000642A0430F0007F2ADC3071020319752A87
:1014D000B23071020319752A2608073A0319732AD4
:1014E000793A031D832D0630762A083070078A1159
:1014F0009A278A150139031D832D1030F00098308A
:10150000832D1530FA009230F900C230F700CF3049
:10151000F6001B21F606F70B892AF60803192E158B
:10152000832D61088400831730300002031C832D53
:101530003A3000020318832D15306402031DB02ACF
:101540002D08DD0000080F39AD00E50122308400D0
:101550008A119B218A155D08AD001530E300E72B49
:1015600016306402031DB72A1630E300E72B28214A
:101570006108823E840045308000840A4E3080003D
:10158000FB2B2D08DD0020308400831700080F3965
:10159000AD008A11A6215D08AD00BD080319BD0A82
:1015A00011303D0201300318BD003D08FB00DF266D
:1015B0004E21223084000008FB008A11DF264E21D4
:1015C0008A15840ABD0BDB2A832D6408E3002821D9
:1015D000A03084003D08FB0020210318212BA030FF
:1015E00084008A1145268A150318212B3D0AE1073C
:1015F0006408163A03191E2B0A3A03191E2BD23A15
:101600000319132B013A0319132B1F3A03190B2B40
:10161000013A031D832D0C30FA00CB30F900640829
:10162000FB002E1615290C30FA00CA30F9006408A8
:10163000FB00CC30E3002D08E4001529CB30E3009B
:10164000832DC930E300412B163A03193F2B013A91
:1016500003193F2B0F3A03193F2B013A03193F2B74
:10166000053A03193F2BD23A03193F2B013A0319CC
:101670003F2B1F3A03193F2B013A031D832DC8301E
:10168000E3000230F300A626803ACA300319E300D3
:101690009B2BD93A0319642B033A0319642BCB3AD9
:1016A0000319642B033A0319642B013A0319642BC1
:1016B000C63A0319642BE23A0319642BE43A03197E
:1016C000642B3F3A031D832DA03084007708BD00B2
:1016D0001B218000840ABD0B682BE50803198E2BA3
:1016E0006108E000A13084000008A23EE200650825
:1016F000F6002E21A13084000008A13EE20065081A
:101700008007840A840A00080407F60062060319A9
:101710008C2B76088400812B65088007A03084001C
:1017200077086507BD0000088A11BC208A1541258D
:10173000BD0B932BE5010315832D6308FE3A0319B6
:10174000A72BFF3A0319A72B1A3A031D832DC1308B
:101750008400D0300002031D840390230800DE3A89
:101760000319BB2BCB3A0319BB2B033A0319BB2B31
:10177000013A031D832D28216308163A031DCB2B44
:101780008030610784008A1163268A150318EA2BCA
:10179000DD30E300E72BCB3A031DD92B8030610706
:1017A00084008A1171268A150318EA2BDE30E300C3
:1017B000E72B8030610784003D08FB0020210318DF
:1017C000EA2BDE306302031DED2BDF30E3003D0A20
:1017D000E1079B2B3D08E5009B2B2821203061026F
:1017E0003D07FD2B28216108833E84005330800093
:1017F000840A4D3080009F300402FC008A1180244E
:101800008A159B2B28216108843E8400413080008A
:10181000840A44308000FB2B013A0319122CE23A6F
:10182000031D832D28218030610784003D08FB00C3
:1018300020210318EA2B19306302031DED2BFB3026
:10184000E300E72B03170830FA00A630F9001B214C
:10185000FB001B21FC00FA01F901A001A101B0303D
:101860001121A10A0A302102031D382CA00AA1016E
:101870007B087A06031D2F2C7C087906031D2F2C6C
:101880002F30A2000830FA008E30F9001B21FB0037
:101890001B21FC00FA01F901A301A401A5012030DC
:1018A0001121A50A0A302502031D582CA40AA501FE
:1018B0000A302402031D5E2CA30AA4017B087A06C9
:1018C000031D4F2C7C087906031D4F2C3030A007D8
:1018D000A107A307A407A50703131230FA00D0300D
:1018E000F9002630840083170D30F7001B2180009B
:1018F000840AF70B762C0030FA000030F9000A3029
:10190000F7008A117820F6008A15E50176080A3C6E
:1019100077062830031D8F2C8000840AE50A77089B
:101920003A3C80008A11132129218A15FF3A2D3073
:101930000319800076080A3C77062930031DA32C82
:10194000840A8000E50A09301121840AF70B862CED
:101950001D30E507832D0F3A031DB82C0130E3003D
:1019600037250408E500CA24E000C0218A15E22CCE
:10197000013A031D832D37250408E500CB24E00040
:10198000E003E003C0218A153B258316DE0ADE0A48
:101990008312262DCE34D034CB24D03A03199B2B7E
:1019A0007008CA3A0311832D81228A15372504084D
:1019B000E5004430F700CA24CE3A0319E22C113076
:1019C0001121F7023B251D2DCA24CE3A0319EB2C19
:1019D000CD30E300832D37250408E5002D08DD0018
:1019E0000A30BD003D080A3CAD000730AC21132190
:1019F00029218A15FF3A0319192D0F30800041253E
:101A00008A11A6218A151B21F700023E800041257C
:101A10002D080A3E800041252D3080005D082D06EE
:101A20002B300319800041251B2180004125F70B35
:101A3000142DBD0BF22C5D08AD00703004020318AC
:101A4000232D2030252D4030831B8402650804029D
:101A5000E500C330831304028402840380008039CC
:101A6000031D832D8403D0308000E5039B2BBE2112
:101A70008A15C03084001B2180004125F70B3B2DC7
:101A80000800840A04087039703A2030031D4A2D7A
:101A90008407831708002E19512D30307402031C5F
:101AA000832D1721F40B512D0314832DBE010C300F
:101AB000F7008A117C208A1502303A02031D622D3C
:101AC0001721F4037408F0390F3003197408F70074
:101AD0000C30F4027702F402F700F7088A11031DB4
:101AE0007E208A15F4080319832DBD033D08F700F5
:101AF000792D61088400831717218000840AF70B71
:101B00007C2D2030800083138A110800FF30AD1B2C
:101B1000AD00EE25FC25DA217820F600FF3A031906
:101B20009828F61F98288030F606F7008A15D225E7
:101B30009828AC250319832D1030FA00F901FB0118
:101B400015210800AC250319832D1030FA00F90186
:101B50006630FB00152108002130BF218A15770867
:101B6000543EF600FF30F7001B21F707F60BB42DAB
:101B7000F7080800EE25FC252D08F6008030F70058
:101B8000263071020319C72DFF30F600F701D22568
:101B900098288A117820F600FF3A0319080080304F
:101BA000F604F7010830FA000E30F9008A11D02649
:101BB0008A15F706F71BE02D0830F0007F22A328D6
:101BC0008030FB068A11DF261E30F900DF26FA017D
:101BD0007830F9007608FB00DF2608008A1108300B
:101BE0007402031D862879208A150830F7005F26C5
:101BF000A626B526842608008330FB060319032E8B
:101C0000FB0015218A1508008A1110307402031D8B
:101C1000862879208A151030F7005F26A926B52678
:101C2000F3080319162EF430F800242EC830F800FB
:101C30000A30F000FF302D020319262EC830F900BB
:101C4000043024217908F8000130F000A926BB26D1
:101C5000A01BA328FF302D02031D312E70080A3C63
:101C6000AD008A30FB0015218A15432E8A111030F1
:101C70007402031D862879208A151030F7005F262C
:101C8000A626B5268426F3080319492EF030F8005D
:101C90004F2EA030F900043024217908F8000430D8
:101CA000F5003430840000088A11BD268A15F80A30
:101CB000840AF50B532EB026233EF9008A2D8A1193
:101CC0007C208A151030F500303084000F308005FC
:101CD000840AF50B672E300E3104B000320E330447
:101CE000B100340E3504B200360E3704B300380E9E
:101CF0003904B4003A0E3B04B5003C0E3D04B60076
:101D00003E0E3F04B7000800F30803198A2EF03096
:101D1000F800982EA030F8000A30F000FF302D02B5
:101D200003199A2EA030F900043024217908F80014
:101D30000130F000A626BB26A01BA328FF302D02F1
:101D4000031DA52E70080A3CAD000800B026233EF6
:101D5000AB2EB026243EF9008A11D0268A15080041
:101D60000830FA00731073080800803A031D080059
:101D7000D4268A11A3280430F50030308400A01343
:101D80008A11B2268A150006031DA017840AF80AD4
:101D9000F50BC02EA01F0800F00BBB2EFB03152176
:101DA0000430F0007B080F3940300319F000983000
:101DB00008008A112608F4228A15043A031DE22E2F
:101DC000F003F0030830FA007007F9008A11D026FA
:101DD0008A150130711F0301FB06031DF12E7D22C0
:101DE000A328FB008A11DF269828A030F9070318E2
:101DF000FA0A9830FA07DC30710203190B2F8A11A6
:101E000079208A11D0267B08BC204E218A15F40B3C
:101E1000012F8A11982819278A15A03084000008FC
:101E2000FB0015214E21840A8A15F40B0F2F8A110D
:101E300098287408F700A03084008A1179208A1548
:101E400017218000840AF70B202F842D8A112F0878
:101E5000F9002708FA0030084D2131084D21790892
:101E6000AF007A08A70008008A112F08F900270898
:101E7000FA0070084D2171084D2172084D21730838
:101E80004D2174084D217908AF007A08A700080099
:101E9000FF3FFF3FFF3FFF3FFF3FFF3FFF3FFF3F52
:101EA000FF3FFF3FFF3FFF3FFF3FFF3FFF3FFF3F42
:101EB000FF3FFF3FFF3FFF3FFF3FFF3FFF3FFF3F32
:101EC000FF3FFF3FFF3FFF3FFF3FFF3FFF3FFF3F22
:101ED000FF3FFF3FFF3FFF3FFF3FFF3FFF3FFF3F12
:101EE000FF3FFF3FFF3FFF3FFF3FFF3FFF3FFF3F02
:101EF000FF3FFF3FFF3FFF3FFF3FFF3FFF3FFF3FF2
:101F0000FF3FFF3FFF3FFF3FFF3FFF3FFF3FFF3FE1
:101F1000FF3FFF3FFF3FFF3FFF3FFF3FFF3FFF3FD1
:101F2000FF3FFF3FFF3FFF3FFF3FFF3FFF3FFF3FC1
:101F3000FF3FFF3FFF3FFF3FFF3FFF3FFF3FFF3FB1
:101F4000FF3FFF3FFF3FFF3FFF3FFF3FFF3FFF3FA1
:101F5000FF3FFF3FFF3FFF3FFF3FFF3FFF3FFF3F91
:101F6000FF3FFF3FFF3FFF3FFF3FFF3FFF3FFF3F81
:101F7000FF3FFF3FFF3FFF3FFF3FFF3FFF3FFF3F71
:101F8000FF3FFF3FFF3FFF3FFF3FFF3FFF3FFF3F61
:101F9000FF3FFF3FFF3FFF3FFF3FFF3FFF3FFF3F51
:101FA000FF3FFF3FFF3FFF3FFF3FFF3FFF3FFF3F41
:101FB000FF3FFF3FFF3FFF3FFF3FFF3FFF3FFF3F31
:101FC000FF3FFF3FFF3FFF3FFF3FFF3FFF3FFF3F21
:101FD000FF3FFF3FFF3FFF3FFF3FFF3FFF3FFF3F11
:101FE000FF3FFF3FFF3FFF3FFF3FFF3FFF3FFF3F01
:101FF000FF3FFF3FFF3FFF3FFF3FFF3FFF3FFF3FF1
:102000006634B134BA34A23402349C3470344B3464
:102010003734193408340C34FB34C134F634BC344E
:102020006D34D534973435342A344F34BF34733457
:10203000E934F234A434DF34D13494346C34A13430
:10204000FC342534F4342F344034D3340634ED34A6
:10205000B934A0348B3471344C348A343B34463434
:1020600043341A340D349D343F34B334DD341E34DC
:10207000D6342434A634453498347C34CF34743484
:10208000F734C234293454344734013431340E34F3
:102090005F342334A934153460344E34D734E134FA
:1020A000B634F3341C345C34C934763404344A34E2
:1020B000F834803411340B3492348434F5343034B1
:1020C00095345A34783427345734E6346A34E83453
:1020D000AF3413347E34BE34CA348D348934B034D2
:1020E000FA341B3465342834DB34E3343A341434A2
:1020F0003334B2346234D8348C34163420347934E6
:102100003D346734CB3448341D346E345534D434C4
:10211000B434CC349634B7340F344234AC34C43491
:102120003834C5349E34003464342D349934073443
:102130009034DE34A334A7343C348734D234E734CB
:10214000AE34A5342634F934E0342234DC34E534BA
:10215000D934D034F1344434CE34BD347D34FF34FA
:10216000EF343634A83459347B347A3449349134DA
:102170007534EA348F3463348134C834C034523413
:102180006834AA348834EB345D345134CD34AD3402
:10219000EC345E34693434342E34E434C6340534DB
:1021A0003934FE3461349B348E348534C734AB34D7
:1021B000BB3432344134B5347F346B349334E2343D
:1021C000B834DA34833421344D3456341F342C344B
:1021D00058343E34EE34123418342B349A341734D5
:1021E00050349F3486346F340934723403345B3492
:1021F0001034823453340A34C334F034FD34773429
:1022000013340B34503472342B34013445345E347F
:10221000273412347F3475346134033455342B340D
:102220001B347C34463453342F3447343F340A341F
:102230002F3459344F3404340E343B340B340534CA
:1022400023346B34673444341534563424345B34CB
:1022500055347E34203432346D345E347834063470
:1022600035344F341C342D3463345F3429342234F4
:10227000583444345D3437346E347D346934143426
:102280005A3450344C34603417343C34593440346C
:10229000793438340E344A346534083413344E34C7
:1022A0004C34423468342E346F34323420340334A6
:1022B000273400343A3419345C341634123433344D
:1022C000393441347734743416346D340734563429
:1022D0003B345D343E346E344E3463344D344334D9
:1022E0000C34713457346234663405345834213434
:1022F00026343834173408344B342D340D344B34F1
:102300005F343F341C3431347B34783414347034CB
:102310002C341E340F3462346A34023467341D3472
:1023200052346B342A347C3418341E34293410343B
:102330006C346434753428344934283407347234A6
:1023400052347334243470340C346634643454346A
:102350005C343034483461340934363437344A34E8
:1023600071347B3411341A3435343A34043409343A
:1023700045347A34153476342A343C341B344934A9
:1023800076347D3422340F34413473345434403441
:102390003E3451344634013418346F347934533474
:1023A0006834513431347F34303469341F340A3462
:1023B00006345B34573425341034363474347E3468
:1023C0001F3426340D34003448346A344D343D34DF
:1023D0001A3443342E341D34603425343D343434BF
:1023E000653411342C346C34473434344234393449
:1023F0002134333419345A34023477347A34233460
:10240000343432342C3406341534313429343B34EA
:10241000273433341934203433342F3434342B34C8
:1024200025340434283422343D340C341C34043430
:102430003A34173408340F340C3416340934123457
:1024400037340A3421342334323401342B34033406
:1024500039340D343E340E3407342A342C343B34B2
:102460003E3439341B34063408341F341A343634BD
:10247000293416342D3414342734033410343834CA
:102480003034023415341C3424342A343C3421349E
:102490002234123400340B3418340A3411343D34ED
:1024A0001D340E342D341A3437342E340B34113499
:1024B00036342E34093418341E343C34203400347D
:1024C0001434263402341E343A34233401341034A4
:1024D00038342834173430340D34133413341B3467
:1024E0001F3435342F3426343F340F34313405341F
:1024F00025343534193424343F341D34053407343D
:10250000013405341D3406341934013412341734BF
:1025100011341334003409341834193406341F3498
:102520001C34143418341E3404341B3403340D3476
:102530000F3410340E3412340434033408340934A4
:10254000143400340C341A34153408341C34023476
:102550001D3402340F3407340B3416340E340A346D
:10256000113415340C341E341A341B3410341F3417
:102570000B3407340D3417340A340534163413344D
:10258000FC34A4341E34B7345034E7341234D83415
:10259000A33449346034323456348934BD34FC3485
:1025A00020344134633474346934763465342034EF
:1025B0004E34723473343A342034D03481345C3441
:1025C00001340334FE3425340034023402348134BF
:1025D000823405340D34533469346D342D3445342C
:1025E0006D347534203436342E3430343134FF3485
:1025F0000F340F340134533465346C342E3450347A
:1026000068346F346E34653420342334FF34FF343F
:10261000FF340F340F34023443346F346E34663475
:1026200069346734753472346534FF34FF34FF34F1
:10263000FF34FF340F340F34033449346E346634BE
:102640006F3472346D346134743469346F346E3481
:10265000FF34FF34FF340F340F3404345234653404
:10266000733465347434FF34FF34FF34FF34FF3483
:10267000FF34FF34FF34FF34D03481341934013453
:10268000033401342434003402340234813482347B
:1026900005340E34533465346C342E34503468347D
:1026A0006F346E34653420342334FF34FF34FF3408
:1026B000D0348134A134013403340234243400345E
:1026C000023402348134823405340E3443346F349E
:1026D0006E34663469346734753472346534FF346B
:1026E000FF34FF34FF34FF340F340F3415344534D6
:1026F00064346934743420342334FF34FF34FF34B9
:10270000FF34FF34FF34FF34FF340F340F341634FA
:1027100043346F346E346634693467342E34503445
:102720006F3473342E34FF34FF34FF340F340F34DE
:10273000173443346F346E346634693467342E345E
:1027400053344D345334FF34FF34FF34FF340F34EB
:102750000F34183443346F346E346634693467345C
:102760002E34413444344E34FF34FF34FF34FF34CC
:102770000F340F341934503449344E3432342F343A
:10278000503455344B343234FF34FF34FF34FF348B
:10279000FF340F340F341A34533465346C342E3410
:1027A000503468346F346E34653420342334FF344D
:1027B000FF34FF340F340F341B344C346F34613426
:1027C000643465347234FF34FF34FF34FF34FF3433
:1027D000FF34FF34FF340F340F341C34453472346B
:1027E000613473346534203450346F3473342E3490
:1027F000FF34FF34FF34FF34D03421340134033448
:1028000015342334013402340234813482340D34DB
:102810000F340434503468346F346E3465342034EB
:1028200023343A34FF34FF34FF34FF34FF34FF34B1
:102830001134023401341034173401340434D034E8
:10284000183401340334163423340034023402348F
:10285000813482340D340634043449344D345334D5
:1028600049343A34113402341234123417340134F6
:102870000434D034163401340334DD3423340134C9
:1028800002340234813482340D34043404344B3441
:1028900049343A34113402342034203417340134AA
:1028A0000434D034173401340334DE342334003498
:1028B00002340234813482340D340534043450340B
:1028C00055344B343A341134023408340834173454
:1028D00001340434D034173401340334DF34233466
:1028E000003402340234813482340D34053404342B
:1028F000503449344E343A341134023404340834F8
:10290000173401340434D034173401340334173409
:102910002334003402340234813482340D340834D8
:1029200004344E3472342E3453344D3453343A34E8
:102930001134023402340234D034173401340334F5
:1029400018342334003402340234813482340D3498
:10295000083404344E3472342E34413444344E340A
:102960003A341134023403340334D034183401348B
:102970000334193423340034023402348134823471
:102980000D3406340434503455344B3432343A3434
:102990001134023408340834173401340434D03488
:1029A000213401340334FB34233400340234023440
:1029B000813482340D340F3404344E34653477342A
:1029C0002034503449344E3432343A34FF34FF34F6
:1029D000FF34FF34FF341134023404340834173424
:1029E00001340434D03481341934013403341B34B9
:1029F00024340034023402348134823405340E34F9
:102A00004C346F346134643465347234FF34FF34D1
:102A1000FF34FF34FF34FF34FF34FF34D0345D34EF
:102A20000134033403342434003402340234813456
:102A3000823405340E3449346E3466346F34723463
:102A40006D346134743469346F346E34FF34FF3460
:102A5000FF340F340F341F3441346334743475340D
:102A600061346C3420344E3472342E34FF34FF34ED
:102A7000FF34FF340F340F34203443346F346E345A
:102A8000663469346734753472346134743469344B
:102A90006F346E34FF340F340F34213456346534C0
:102AA0007234733469346F346E34FF34FF34FF345E
:102AB000FF34FF34FF34FF340F340F3422344134F9
:102AC0007534743468346F347234FF34FF34FF3437
:102AD000FF34FF34FF34FF34FF34D0340C3401347E
:102AE00003341F34213481340234023481340234FB
:102AF0000D3401340434D03415340134033420341B
:102B00002134813402340234813402340D340A34E5
:102B1000043453344D3453342F34413444344E341C
:102B20003A342034E6345D343134303413341C34D8
:102B3000BD343D343C34B8343A3436345B3401343B
:102B400057346E346B342C3445346E3477342D3432
:102B50003A3421343E343834283423343A3423345C
:102B60003B3425342634213423343A34323430345F
:102B70003C344B34763470346B343B3469340A342F
:102B800002341334113400341234063442340E3417
:102B90000D340134003406341C344B340834103402
:102BA0005434043419341D34143453341C3418345C
:102BB00015340B3416341C340A345B3413342B3480
:102BC00027342B34333425342534273462342434E9
:102BD00022346F342F34273431346B3429343A346F
:102BE00039343A343334233433343A3433343134AB
:102BF0007C342F342C3436343C342E343934D134B4
:102C00007434F534A734A234823482342334AF349C
:102C1000AE342E34AC34A434EF34AF34EE34D43488
:102C2000DA34DE34D334DD349034F934D334DF3461
:102C3000D534D9349E3494349834EC34DF34E734CA
:102C4000BE34A734EE34F534F434F334B834A2345B
:102C5000A334FC34E734E434ED34E634FF34BB34DD
:102C6000F734FD34F434BF34FE34F634E634BD3486
:102C7000B134BF34DB34F434F934F234F634DF34B5
:102C8000C4348E34883487348F34E33491348434BC
:102C900081348A3483349C34C63488348034973405
:102CA000DA34993493348534D0340934013403341C
:102CB0000434013404340234023481348234D03494
:102CC000153401340334C834233404340234023458
:102CD000813482340D3406340434503449344E3453
:102CE00032343A341134023404340834D0341B34CE
:102CF00001340334C9342134813402340234813440
:102D000002340D341034043449346E347634613472
:102D10006C34693464342034503449344E343234A1
:102D2000FF34FF34FF34D0341A3401340334CA344E
:102D30002134813402340234813402340D340F34AE
:102D40000434503449344E34323420346C346F34CB
:102D500063346B3465346434FF34FF34FF34D0346F
:102D60001D3401340334CB342334003402340234B0
:102D7000813482340D340E34043450346F3473345F
:102D80006934743469346F346E343A34FF34FF3448
:102D9000FF34FF341134023401340134D0340934A7
:102DA00001340334CC34013400340234023481342D
:102DB0008234D0341E3401340334CD342134813490
:102DC00002340234813402340D3413340434443474
:102DD0006534613463347434693476346134743402
:102DE0006534643420346F347034743469346F342F
:102DF0006E340F340E34CE34413463347434693459
:102E00007634613474346534FF34FF34FF34FF3476
:102E1000FF340F340E34CF344434653461346334BA
:102E2000743469347634613474346534FF34FF3477
:102E3000FF34FE341234DD341B34013413343C349B
:102E40001C34023413345834A43415341334FC3491
:102E50002334163414341F341A34DD341434393422
:102E60001834DE34143451341934DF3414346A34F1
:102E700019341734143483341934183414349C340A
:102E8000193419341434B5341A34FB341434CF34AF
:102E900023341B341434F2341C34033415340E340C
:102EA0005F341F3415346D340E34203415347B34C4
:102EB00017342134153492346E34223416340034ED
:102EC00054340434163454340B34C83416345F3458
:102ED0001734C934163476341D34CA341634933456
:102EE0001C34CB341634AF341F34CC341634CE34C7
:102EF0000B34CD341634D9342034CF341634F9346D
:102F00001034CE341734093410340734003400340C
:102F10000934203400345A34093437340034B4349A
:102F2000033439340034D2340534413401340434A8
:102F30000534423401343634203474340234763467
:102F400010347E34033416340B3452340334843456
:102F5000093453340334DE340E340034083450342E
:102F600068346F346E346534203423343034203484
:102F700020342034203420342034203420340834C9
:102F8000503468346F346E34653420342334313433
:102F90002034203420342034203420342034203491
:102FA0000834503468346F346E346534203423343C
:102FB000323420342034203420342034203420345F
:102FC00020340834503468346F346E34653420341F
:102FD000233433342034203420342034203420343B
:102FE000203420340834503468346F346E346534FF
:102FF000203423343434203420342034203420341A
:103000002034203420340834503468346F346E3423
:1030100065342034233435342034203420342034B3
:1030200020342034203420340834503468346F3451
:103030006E34653420342334363420342034203444
:103040002034203420342034203408345034683480
:103050006F346E34653420342334373420342034D4
:1030600020342034203420342034203408345034A8
:1030700068346F346E34653420342334383420346B
:1030800020342034203420342034203420340834B8
:10309000503468346F346E3465342034233439341A
:1030A0002034203420342034203420342034203480
:1030B0003F342834003400341134143400340334E1
:1030C00068349034003407343134E23485340534C4
:1030D0002D342034453430344D3431345134373488
:1030E00055343834593441345D34433461344534D3
:1030F000653452346D345334713474344934783413
:1031000075347B3479347E343B34AD347D34AE3425
:1031100081343934ED343D34B1344034BD3442343B
:10312000C9344434E134463469344A34D5343B3408
:1031300099343C34A534073489343A348D3400341E
:10314000FF3FFF3FFF3FFF3FFF3FFF3FFF3FFF3F8F
:10315000FF3FFF3FFF3FFF3FFF3FFF3FFF3FFF3F7F
:10316000FF3FFF3FFF3FFF3FFF3FFF3FFF3FFF3F6F
:10317000FF3FFF3FFF3FFF3FFF3FFF3FFF3FFF3F5F
:02400E00292F58
:10420000FF00FF00FF00FF00FF00FF00FF00FF00B6
:10421000FF00FF00FF00FF00FF00FF00FF00FF00A6
:10422000FF00FF00FF00FF00FF00FF00FF00FF0096
:10423000FF00FF00FF00FF00FF00FF00FF00FF0086
:10424000FF00FF00FF00FF00FF00FF00FF00FF0076
:10425000FF00FF00FF00FF00FF00FF00FF00FF0066
:10426000FF00FF00FF00FF00FF00FF00FF00FF0056
:10427000FF00FF00FF00FF00FF00FF00FF00FF0046
:10428000FF00FF00FF00FF00FF00FF00FF00FF0036
:10429000FF00FF00FF00FF00FF00FF00FF00FF0026
:1042A000FF00FF00FF00FF00FF00FF00FF00FF0016
:1042B000FF00FF00FF00FF00FF00FF00FF00FF0006
:1042C000FF00FF00FF00FF00FF00FF00FF00FF00F6
:1042D000FF00FF00FF00FF00FF00FF00FF00FF00E6
:1042E000FF00FF00FF00FF00FF00FF00FF00FF00D6
:1042F000FF00FF00FF00FF00FF00FF00FF00FF00C6
:10430000FF00FF00FF00FF00FF00FF00FF00FF00B5
:10431000FF00FF00FF00FF00FF00FF00FF00FF00A5
:10432000FF00FF00FF00FF00FF00FF00FF00FF0095
:10433000FF00FF00FF00FF00FF00FF00FF00FF0085
:1043400000000000FF00FF0011001100FF00FF004F
:1043500022002200FF00FF00FF00FF00FF00FF001F
:10436000FF00FF00FF00FF00FF00FF00FF00FF0055
:10437000FF00FF00FF00FF00FF00FF00FF00FF0045
:10438000FF00FF00FF00FF00FF00FF00FF00FF0035
:1043900000000000000000001100110011001100D9
:1043A0002200220022002200FF00FF00FF00FF0089
:1043B000FF00FF00FF00FF00FF00FF00FF00FF0005
:1043C000FF00FF00FF00FF00FF00FF00FF00FF00F5
:1043D000FF00FF00FF00FF00FF00FF00FF00FF00E5
:1043E00012003400FF00FF00120034005600780075
:1043F000FF00FF00FF00FF00FF00FF00FF00FF00C5
:00000001FF
